:100000000C94BA000C94F8070C941D080C94E200B0
:100010000C94E2000C94E2000C94E2000C94E200D8
:100020000C94E2000C94E2000C94E2000C94E200C8
:100030000C94E2000C94E2000C94E2000C94E200B8
:100040000C94AE070C94E2000C947C070C945607B9
:100050000C94E2000C94E2000C94E2000C94E20098
:100060000C94E2000C94E200FF0408051305C2059D
:1000700032053B05C205C205C205C205C205C2055F
:10008000C205C20545055805C205C205C205C2051F
:1000900087058F0592059E05B805380C360C3D0C7A
:1000A000540CEE0C760C970CB30CCF0C000DFE0C20
:1000B000050D1C0D1C0D3E0D5F0D7B0D970D0800F1
:1000C0000000BE922449123EABAAAA2ABECDCCCCD7
:1000D0004C3E00000080BEABAAAAAA3E0000000071
:1000E000BF000000803F0000000000084178D3BB43
:1000F0004387D1133D190E3CC3BD4282AD2B3E68F0
:10010000EC8276BED98FE1A93E4C80EFFFBE01C4E0
:10011000FF7F3F00000000000000000024002700D7
:100120002A0000000000250028002B00000000002D
:100130002300260029000404040404040404020229
:100140000202020203030303030301020408102056
:100150004080010204081020010204081020000061
:100160000008000201000003040700000000000076
:100170000000D90E11241FBECFEFD8E0DEBFCDBFE7
:1001800022E0A0E2B1E001C01D92AC33B207E1F77A
:1001900011E0A0E0B1E0E4E5F4E202C005900D92C8
:1001A000A032B107D9F710E0CAEBD0E004C0219724
:1001B000FE010E94060FC93BD107C9F70E94420801
:1001C0000C9428120C940000CF92DF92EF92FF92D1
:1001D0006B017C01E091AF01F091B00182E080837E
:1001E000C11481EED806E104F104B1F060E079E0D9
:1001F0008DE390E0A70196010E94F711DA01C90191
:100200000197A109B109B695A795979587959C0186
:10021000211580E13807B8F0E091AF01F091B0010D
:10022000108260E874E88EE190E0A70196010E94D8
:10023000F711DA01C9010197A109B109B695A7958E
:10024000979587959C01E091AB01F091AC013083CB
:10025000E091AD01F091AE0120831092B701E091E1
:10026000B301F091B40186E08083E091B101F09197
:10027000B201808180618083E091B101F091B2018F
:10028000808188608083E091B101F091B20180812A
:1002900080688083E091B101F091B20180818F7D0F
:1002A0008083FF90EF90DF90CF900895CF92DF9200
:1002B000EF92FF920F931F93CF93DF936C017A011C
:1002C0008B01C0E0D0E0CE15DF0589F0D8016D913B
:1002D0008D01D601ED91FC910190F081E02DC601D8
:1002E0000995892B11F47E0102C02196ECCFC7013C
:1002F000DF91CF911F910F91FF90EF90DF90CF9002
:100300000895FC01918D828D981761F0828DDF0137
:10031000A80FB11D5D968C91928D9F5F9F73928FF8
:1003200090E008958FEF9FEF0895FC01918D828DED
:10033000981731F0828DE80FF11D858D90E00895BA
:100340008FEF9FEF0895FC01918D228D892F90E012
:10035000805C9F4F821B91098F7399270895CF93DB
:10036000C1E08FE991E00E94A301892BF9F08FE9A8
:1003700091E00E94810190919E01981307C0C09363
:100380009D0190939901C0939801EBCF90919D01AD
:10039000992339F3E091980191E09E0F9093980191
:1003A000F0E0E756FE4F80839430D8F280919801B8
:1003B000843010F480E01DC09091990190939401D5
:1003C00030919A013093950180919B018093960121
:1003D00020919C0120939701930F890F982F9F776D
:1003E00081E0921380E01092990110929D01109289
:1003F0009801CF9108958FE991E00E94A30121E037
:10040000892B09F420E0822F0895FC01848DDF01FF
:10041000A80FB11DA35ABF4F2C91848D90E0019677
:100420008F739927848FA689B7892C93A089B18966
:100430008C9180648C93938D848D981306C0028870
:10044000F389E02D80818F7D80830895EF92FF9264
:100450000F931F93CF93DF93EC0181E0888F9B8DE7
:100460008C8D981305C0E889F989808185FD24C0A9
:10047000F62E0B8D10E00F5F1F4F0F731127E02E2C
:100480008C8DE8120CC00FB607FCFACFE889F98909
:10049000808185FFF5CFCE010E940502F1CF8B8DC3
:1004A000FE01E80FF11DE35AFF4FF0820B8FEA893E
:1004B000FB898081806207C0EE89FF896083E889BB
:1004C000F98980818064808381E090E0DF91CF9121
:1004D0001F910F91FF90EF900895CF93DF93EC0160
:1004E000888D8823C9F0EA89FB89808185FD05C054
:1004F000A889B9898C9186FD0FC00FB607FCF5CF8E
:10050000808185FFF2CFA889B9898C9185FFEDCFD5
:10051000CE010E940502E7CFDF91CF91089580E0E0
:1005200090E0892B29F00E94FB0181110C940000BE
:100530000895833081F028F4813099F08230A1F061
:1005400008958730A9F08830B9F08430D1F48091D3
:1005500080008F7D03C0809180008F778093800022
:10056000089584B58F7702C084B58F7D84BD0895CA
:100570008091B0008F7703C08091B0008F7D809311
:10058000B0000895CF93DF93282F30E0F901E25AAD
:10059000FE4F8491F901E65BFE4FD491F901EA5CCC
:1005A000FE4FC491CC2391F081110E949902EC2F4F
:1005B000F0E0EE0FFF1FE45DFE4FA591B491EC91CA
:1005C000ED2381E090E021F480E002C080E090E043
:1005D000DF91CF9108951F93CF93DF93282F30E0C1
:1005E000F901E25AFE4F8491F901E65BFE4FD49186
:1005F000F901EA5CFE4FC491CC23C9F0162F81119A
:100600000E949902EC2FF0E0EE0FFF1FEE5DFE4F0F
:10061000A591B4918FB7F894111105C09C91ED2F5D
:10062000E095E92302C0EC91ED2BEC938FBFDF91B5
:10063000CF911F910895CF93DF9390E0FC01E65B8B
:10064000FE4F2491FC01EA5CFE4F8491882361F106
:1006500090E0880F991FFC01E85EFE4FC591D49190
:10066000FC01EE5DFE4FA591B491611109C09FB7E9
:10067000F8948881209582238883EC912E230BC0E7
:10068000623061F49FB7F8943881822F809583237C
:100690008883EC912E2B2C939FBF06C08FB7F894C4
:1006A000E8812E2B28838FBFDF91CF9108958E3064
:1006B00008F08E508770806480937C0080917A006F
:1006C000806480937A0080917A0086FDFCCF8091CF
:1006D00078002091790090E0922B08953FB7F8942C
:1006E0008091350190913601A0913701B091380188
:1006F00026B5A89B05C02F3F19F00196A11DB11D7D
:100700003FBFBA2FA92F982F8827820F911DA11DB7
:10071000B11DBC01CD0142E0660F771F881F991FF4
:100720004A95D1F708958F929F92AF92BF92CF9240
:10073000DF92EF92FF926B017C010E946E034B01EE
:100740005C01C114D104E104F104F1F00E946E03D4
:10075000DC01CB0188199909AA09BB09883E93409D
:10076000A105B10570F321E0C21AD108E108F10832
:1007700088EE880E83E0981EA11CB11CC114D10420
:10078000E104F10419F7DDCFFF90EF90DF90CF90F7
:10079000BF90AF909F908F9008952FB7F89460917D
:1007A00031017091320180913301909134012FBF5A
:1007B00008958F929F92AF92BF92CF92DF92EF9265
:1007C000FF9284E10E945703BC01990F880B990B9B
:1007D0000E94211020E030E040E85AE30E942611F8
:1007E00020E030E040EA50E40E9426116B017C01D9
:1007F00080910001882351F0C0922C01D0922D01EC
:10080000E0922E01F0922F011092000126E636E6CA
:1008100046E65FE360912C0170912D0180912E01DD
:1008200090912F010E9426114B015C0120ED3CECC0
:100830004CEC5DE3C701B6010E9426119B01AC019F
:10084000C501B4010E940D0F60932C0170932D011E
:1008500080932E0190932F012DE33CE248E450E475
:100860000E94261120E030E0A9010E940D0FFF90A8
:10087000EF90DF90CF90BF90AF909F908F900895B2
:1008800085E00E94C20261E0892B09F060E085E00A
:100890000E94EB0287E00E94C20261E0892B09F00E
:1008A00060E087E00E94EB0284E00E94C20261E007
:1008B000892B09F060E084E00E94EB0280E10E9455
:1008C000C20261E0892B09F060E080E10C94EB0248
:1008D00061E084E00E94EB0261E080E10C94EB02B5
:1008E00061E085E00E94EB0261E087E00C94EB029E
:1008F00010928E0110928D01109289001092880042
:100900008091910181110C946804089510929001D6
:1009100010928F0110928B0010928A0080919101A9
:1009200081110C9470040895CF93DF93EB011C1692
:100930001D0684F4813031F461E085E00E94EB0211
:1009400060E011C08230E1F561E084E00E94EB02DA
:1009500060E014C02097B1F0813049F460E085E098
:100960000E94EB0261E087E00E94EB021BC0823034
:1009700039F560E084E00E94EB0261E080E10E94D2
:10098000EB0220C090919101992351F0813019F42C
:100990000E94700407C0823011F50E94680412C0E2
:1009A000813071F4D0939001C0938F01D7FF03C0C1
:1009B000D195C195D109D0938B00C0938A000FC007
:1009C000823069F4D0938E01C0938D01D7FF03C0AC
:1009D000D195C195D109D0938900C0938800DF914A
:1009E000CF910895E09195018E2F90E08931910586
:1009F00008F0C8C0FC01EC5CFF4F0C94060F60913E
:100A0000960167FD6FE723E0629FB001112408C0E3
:100A10006091960167FD6FE72DEF2603B001112469
:100A200081E00C94940460919601633308F0AAC0AD
:100A300070E080E090E00E941F102DEC3CEC4CE454
:100A40005EE30E94261120E030E040EC50E40E947A
:100A50000D0F609307017093080180930901909333
:100A60000A0108956091960167FD6FE783E0689F32
:100A7000B001112408C06091960167FD6FE72DEF6A
:100A80002603B001112482E0CCCF80919601811120
:100A900003C010929301089524E6829FC00111249F
:100AA000909306018093050181E08093930108955E
:100AB000809196018330B9F028F4813049F082307A
:100AC00061F008958530C9F098F08630D9F0089526
:100AD00060E679E080E090E004C060E875E280E0E4
:100AE00090E00C94E40060E07BE480E090E0F9CFDB
:100AF00060E076E980E090E0F4CF60E072EC81E0C5
:100B000090E0EFCF60E071EE80E090E0EACF80917E
:100B100096018093B30081E0809392010895109232
:100B200092010895809196019FEF980F9E3150F5A4
:100B300090E09093040180930301089580919601C1
:100B4000882399F081E08093910180918F019091A9
:100B50009001892B11F40E94700480918D01909175
:100B60008E01892B79F40C946804109291010895F8
:100B700080919601882321F081E080938C01089573
:100B800010928C010895CF92DF92EF92FF920F9313
:100B90001F93CF93C82F0E946E03C11114C04B9BAB
:100BA00009C06093240170932501809326019093DE
:100BB0002701D0C000912401109125012091260128
:100BC0003091270116C0C13009F0C4C04A9B09C04A
:100BD000609328017093290180932A0190932B013F
:100BE000B9C0009128011091290120912A0130916A
:100BF0002B016B017C01C01AD10AE20AF30A9701AA
:100C000086014C2F50E0E0E2CE1AE3E0DE0AE10874
:100C1000F108E9E7CE16E5E0DE06E104F10408F0AC
:100C200069C0FA01EE0FFF1FEE0FFF1FEF59FE4FD5
:100C30006083718382839383FA01EE5DFE4F80812E
:100C40008130B1F0823019F0811175C005C0108279
:100C5000FA01E05EFE4F09C0DA01A05EBE4F8C9142
:100C60008F5F8C93853008F466C081E0808363C019
:100C7000CF5FD901C801875D9540A109B1090B97E4
:100C8000A105B10558F4C13019F40E94860453C07F
:100C9000C23009F050C00E9478044DC0083E83E085
:100CA00018072105310538F0013DE7E01E0728F05F
:100CB00000ED17E002C008EE13E0C801A0E0B0E0CC
:100CC0009C01AD01285E334041095109AAEFB2E011
:100CD0000E94EC1128EE33E040E050E00E94CD117C
:100CE000CA01B9016D577140810991098C2F0E9489
:100CF000940421C0FA01EE0FFF1FEE0FFF1FEF5902
:100D0000FE4F0081118122813381DC01CB01801BE8
:100D1000910BA20BB30B813A9648A140B10558F054
:100D2000FA01EE5DFE4F82E08083FA01E05EFE4F45
:100D30001082CF5FA8CF8091220190912301891763
:100D400039F0813011F0913011F481E001C082E07E
:100D500080936D01CF911F910F91FF90EF90DF90E5
:100D6000CF9008958DE00E94C20261E0892B09F0C6
:100D700060E08DE00C94EB0281E10E94C20261E030
:100D8000892B09F060E081E10C94EB02CF92DF92B5
:100D9000EF92FF92CF93DF93EC010E94CD036B01A2
:100DA0007C018B819C81AD81BE81B701A601481B6E
:100DB000590B6A0B7B0B8F819885A0E0B0E08417FC
:100DC0009507A607B70708F58A8180FD02C061E094
:100DD00001C060E088810E94EB0288EC90E0988777
:100DE0008F83CB82DC82ED82FE828A818F5F8A8351
:100DF000298190E030E0220F331F8217930729F4F6
:100E000088EE93E098878F831A82DF91CF91FF90CD
:100E1000EF90DF90CF9008950E94C8118FE00E945C
:100E20005703BC01990F880B990B0E9421109B015D
:100E3000AC0160E070EC8FE794E40E947E0F20E04C
:100E400030E040E85FE30E940C0F9B01AC0160E0E2
:100E500070E48CE196E40E947E0F20E030E44CE1E7
:100E600056E40E947E0F0E94DE1020E030EF47E53E
:100E700055E40E947E0F2FE03FEC4BE55BE30E94C0
:100E80000D0F9B01AC0160E070E080E89FE30E94E1
:100E90007E0F23E333E948E853E40E940C0F0E94DD
:100EA000F00F709386016093850108951F920F9251
:100EB0000FB60F9211242F933F934F935F936F932D
:100EC0007F938F939F93AF93BF93EF93FF938FE99C
:100ED00091E00E940502FF91EF91BF91AF919F9128
:100EE0008F917F916F915F914F913F912F910F90D3
:100EF0000FBE0F901F9018951F920F920FB60F9272
:100F000011242F938F939F93EF93FF93E091AF0161
:100F1000F091B0018081E091B501F091B60182FDC0
:100F200012C090818091B8018F5F8F732091B901B9
:100F3000821751F0E091B801F0E0E156FE4F958F35
:100F40008093B80101C08081FF91EF919F918F91B3
:100F50002F910F900FBE0F901F9018951F920F9218
:100F60000FB60F9211242F933F938F939F93AF93BC
:100F7000BF938091310190913201A0913301B091E2
:100F800034013091300123E0230F2D3720F40196F6
:100F9000A11DB11D05C026E8230F0296A11DB11D9C
:100FA000209330018093310190933201A09333015B
:100FB000B09334018091350190913601A0913701B1
:100FC000B09138010196A11DB11D80933501909318
:100FD0003601A0933701B0933801BF91AF919F9133
:100FE0008F913F912F910F900FBE0F901F901895EA
:100FF0001F920F920FB60F9211242F933F934F938E
:101000005F936F937F938F939F93AF93BF93EF9370
:10101000FF9381E00E94C305FF91EF91BF91AF91D3
:101020009F918F917F916F915F914F913F912F9100
:101030000F900FBE0F901F9018951F920F920FB632
:101040000F9211242F933F934F935F936F937F934E
:101050008F939F93AF93BF93EF93FF9380E00E9492
:10106000C305FF91EF91BF91AF919F918F917F91B8
:101070006F915F914F913F912F910F900FBE0F9005
:101080001F901895CF93DF9300D000D0CDB7DEB777
:10109000789484B5826084BD84B5816084BD85B553
:1010A000826085BD85B5816085BD80916E0081605F
:1010B00080936E0010928100809181008260809305
:1010C0008100809181008160809381008091800007
:1010D0008160809380008091B10084608093B10032
:1010E0008091B00081608093B00080917A0084602C
:1010F00080937A0080917A00826080937A00809158
:101100007A00816080937A0080917A008068809371
:101110007A001092C10061E085E00E941B0361E04B
:1011200087E00E941B0361E08AE00E941B0360E0ED
:101130008EE00E941B0362E088E00E941B0361E0D6
:1011400084E00E941B0361E080E10E941B0361E0D8
:1011500089E00E941B0360E082E10E941B0362E0C1
:1011600083E10E941B0362E08CE00E941B0361E0AC
:101170008BE00E941B0360E08FE00E941B0362E093
:1011800083E00E941B0362E082E00E941B0361E097
:1011900081E10E941B0360E081E10E94EB0261E0BB
:1011A0008DE00E941B0360E08DE00E94EB0281E174
:1011B000809353018DE08093450162E086E00E94B8
:1011C0001B0386E00E94C202892B11F083E801C054
:1011D00084E880939E0160E076E980E090E00E94E0
:1011E000E4001092720110928B0182EA80938000D9
:1011F00081E18093810087E286BB10926F008DE7CA
:1012000091E0909387008093860010928500109261
:101210008400109289001092880010928B00109226
:101220008A0083E88093B00082E08093B10087E079
:1012300087BB109270001092B2001092B30085E04C
:101240008093690083E08DBB8CBB44E0342E53E077
:10125000252E68EC662E712C10918B01111133C173
:101260008CE00E94C202892B21F435E0C32EC0928B
:101270008B010E94CD03009187011091880120917C
:10128000890130918A01DC01CB01801B910BA20BFB
:10129000B30B893C9105A105B105A8F00E940E078A
:1012A0000E94CD0360938701709388018093890128
:1012B00090938A01809185019091860187399105EB
:1012C00010F030928B0188E00E94C202892B09F451
:1012D000E9C483E10E94C202892B09F4E3C40E949D
:1012E000CD03009181011091820120918301309101
:1012F0008401DC01CB01801B910BA20BB30B853663
:101300009105A105B10508F4C7C00E94CD034B01AA
:101310005C016093810170938201809383019093BB
:1013200084018EE00E94570325E2D22ED89E8001D0
:10133000D99E100D112480910201882331F0109361
:10134000400100933F011092020160913F017091B2
:10135000400180E090E00E941F1026E636E646E657
:101360005FE30E9426116B017C01B80180E090E0F0
:101370000E941F1020ED3CEC4CEC5DE30E94261116
:101380009B01AC01C701B6010E940D0F0E94F00F36
:101390006B017C017093400160933F0180910301D8
:1013A0009091040128EE33E0829F2001839F500C2E
:1013B000929F500C11244C145D0430F480913C0138
:1013C0008F5F80933C0102C010923C0182E10E9439
:1013D000570335E2389F8001399F100D1124809109
:1013E0000101882331F010933E0100933D011092DA
:1013F000010160913D0170913E0180E090E00E940A
:101400001F1026E636E646E65FE30E942611698352
:101410007A838B839C83B80180E090E00E941F1048
:1014200020ED3CEC4CEC5DE30E9426119B01AC01ED
:1014300069817A818B819C810E940D0F0E94F00F3F
:1014400070933E0160933D014616570630F420919B
:101450003B012F5F20933B0102C010923B01C60E5F
:10146000D71ED0923A01C092390180913C018B3055
:1014700020F480913B018B3078F010923B01109268
:101480003C0180927D0190927E01A0927F01B092FA
:10149000800141E040938B010E94CD0300917901CE
:1014A00010917A0120917B0130917C01DC01CB010C
:1014B000801B910BA20BB30B853F9140A105B10599
:1014C00008F0F3C3CDC00E9486040E947804133054
:1014D00009F494C03CF4113009F472C0123009F4DC
:1014E000A4C0BEC0143021F0153009F4B0C0B8C09B
:1014F0000E94CD0300917501109176012091770132
:1015000030917801DC01CB01801B910BA20BB30B56
:1015100089389341A105B105F0F00E9486040E942C
:1015200078040E94400468EC70E080E090E00E9443
:1015300093030E94400462E370E080E090E00E9428
:1015400093030E94CD03609375017093760180939D
:101550007701909378010E94CD030091870110914B
:1015600088012091890130918A01DC01CB01801B27
:10157000910BA20BB30B893C9105A105B10560F05D
:101580000E940E070E94CD0360938701709388012B
:101590008093890190938A0188E00E94C20201979A
:1015A00009F0B1C383E10E94C202019709F0ABC305
:1015B000809185019091860186399105B0F0A3C391
:1015C0000E94CD0300917D0110917E0120917F0149
:1015D00030918001DC01CB01801B910BA20BB30B7E
:1015E00089389341A105B10518F010928B0138C0DC
:1015F0001092740146E04093730132C00E94D903F7
:1016000020910701309108014091090150910A0190
:101610000E94D11018160CF07CC30E94CD036938CB
:1016200073418105910508F774C30E94D90320E036
:1016300030E040E851E40E94790F87FF70C30E94B8
:10164000CD03693873418105910578F668C38CE054
:101650000E94C202892B49F63092730110927401E4
:1016600080918B018111F2C01092730180917201FF
:10167000813009F457C0823019F08111E7C0B9C038
:101680000E94AF01882361F00E94F2040E94CD0302
:1016900060936E0170936F0180937001909371015C
:1016A00080919301882329F10E94CD0300916E015E
:1016B00010916F012091700130917101AB01BC015B
:1016C000401B510B620B730B809105019091060139
:1016D000A0E0B0E084179507A607B70728F40E949A
:1016E00086040E94780482C0CC24C394C092740102
:1016F000ADC00E94CD0300916E0110916F01209149
:10170000700130917101DC01CB01801B910BA20BA8
:10171000B30B893E9340A105B10530F332E030931D
:10172000740194C080916D01813049F0823009F4D8
:101730005DC081118BC042E04093740187C08093EB
:1017400074010E94CD030091690110916A012091FA
:101750006B0130916C01DC01CB01801B910BA20B62
:10176000B30B85369105A105B10508F46FC00E9441
:10177000CD036093690170936A0180936B0190932C
:101780006C01F8940E946E03009161011091620156
:1017900020916301309164016B017C01C01AD10A70
:1017A000E20AF30A41EAC41646E8D40641E0E40638
:1017B000F104D0F00091650110916601209167015C
:1017C00030916801DC01CB01801B910BA20BB30BA4
:1017D000813A9648A140B10538F00E9486040E94E3
:1017E0007804F2E0F0936D01789430C02092740197
:1017F0002DC080916D01813029F480937201809316
:10180000740119C00E94AF018823A9F092E0C92E8B
:10181000C09272011DBA0E94F2040E94CD0360932F
:101820006E0170936F018093700190937101DD24BC
:10183000D394D092740180917201811105C082E02D
:10184000E82EE092730102C010927301E0917401DE
:101850008E2FEE0F990BAA0BBB0B8930910508F068
:10186000BDC0FC01E35BFF4F0C94060F61E001C0BB
:1018700060E081E10E94EB02B1C00E94CD030091C3
:101880005D0110915E0120915F0130916001DC01EA
:10189000CB01801B910BA20BB30B8F3E9240A10595
:1018A000B10508F49BC015C00E94CD0300915D01F5
:1018B00010915E0120915F0130916001DC01CB014C
:1018C000801B910BA20BB30B8997A105B10508F4FE
:1018D00085C00E94BC060E94CD0360935D01709399
:1018E0005E0180935F019093600178C080915C01FC
:1018F000882321F0809154018230A1F032E03093AE
:1019000054011092550110925601109257011092F5
:1019100058011092590170925B0160925A0141E0A6
:1019200040935C0183E591E00E94C60657C0809118
:101930005C01882321F080915401833099F3209237
:1019400054011092550110925601109257011092B5
:1019500058011092590170925B0160925A0181E026
:1019600080935C01DFCF80915C01882321F080911E
:1019700054018430B9F23092540110925501109202
:10198000560110925701109258011092590170920D
:101990005B0160925A01E1E0E0935C01C3CF80916A
:1019A0005C01882329F080915401853009F4BACF75
:1019B000F5E0F093540110925501109256011092E7
:1019C0005701109258011092590170925B01609278
:1019D0005A01CC24C394C0925C01A4CFE09173015E
:1019E0008E2FEE0F990BAA0BBB0B8930910508F0D7
:1019F000BDC0FC01EA5AFF4F0C94060F61E001C024
:101A000060E08DE00E94EB02B1C00E94CD03009126
:101A10004F01109150012091510130915201DC0190
:101A2000CB01801B910BA20BB30B8F3E9240A10503
:101A3000B10508F49BC015C00E94CD0300914F0171
:101A4000109150012091510130915201DC01CB01E4
:101A5000801B910BA20BB30B8997A105B10508F46C
:101A600085C00E94B2060E94CD0360934F0170931F
:101A70005001809351019093520178C080914E01A2
:101A8000882321F0809146018230A1F032E030932A
:101A9000460110924701109248011092490110929C
:101AA0004A0110924B0170924D0160924C0141E04D
:101AB00040934E0185E491E00E94C60657C0809194
:101AC0004E01882321F080914601833099F32092C2
:101AD000460110924701109248011092490110925C
:101AE0004A0110924B0170924D0160924C0181E0CD
:101AF00080934E01DFCF80914E01882321F08091A9
:101B000046018430B9F2309246011092470110929A
:101B100048011092490110924A0110924B017092B3
:101B20004D0160924C01E1E0E0934E01C3CF809102
:101B30004E01882329F080914601853009F4BACFFF
:101B4000F5E0F0934601109247011092480110927F
:101B5000490110924A0110924B0170924D0160921E
:101B60004C01CC24C394C0924E01A4CF80918B0130
:101B7000843011F0813029F4DD24DA94D092B3005E
:101B800058C080919201811154C0209185013091FB
:101B9000860128323105C8F027343105C0F4C90167
:101BA000A0E0B0E09C01AD01285231094109510982
:101BB000AFEAB0E00E94EC112EE130E040E050E0EE
:101BC0000E94CD1110E5120F03C010E001C01FEFFD
:101BD00080913F019091400120913D0130913E0163
:101BE0002817390708F49C01203747E13407C8F06B
:101BF000213E8EE23807D0F4C901A0E0B0E09C019C
:101C0000AD012057374141095109AFEAB0E00E94C8
:101C1000EC1120E737E140E050E00E94CD11205B5D
:101C200001C020E0211718F4212F01C02FEF2093CD
:101C3000B30080918C01882391F10E94CD03009123
:101C40004101109142012091430130914401DC0196
:101C5000CB01801B910BA20BB30B0D97A105B10516
:101C6000F0F000918F01109190010115110509F01C
:101C70005CC00E94700400918D0110918E010115CD
:101C8000110509F074C00E9468040E94CD0360939E
:101C900041017093420180934301909344010E945B
:101CA0008F02DACA30928B011ACB0E94D9036B01E2
:101CB0007C010E94CD036093790170937A01809337
:101CC0007B0190937C0120910701309108014091A4
:101CD000090150910A01C701B6010E94790F87FFDF
:101CE00003C020928B01BCCC20E030E040E851E4FE
:101CF000C701B6010E94D11018160CF0B1CCF2E069
:101D0000F0938B01ADCC10927401E5E0E093730188
:101D1000A7CC10927401F7E0F0937301A1CC10925C
:101D2000740188E0809373019BCC980117FF04C075
:101D300022273327201B310B80918D0190918E013A
:101D400097FF03C091958195910905972817390749
:101D50000CF091CF0E94700463E070E080E090E0AE
:101D60000E949303B80181E00E94940484CF9801FB
:101D700017FF04C022273327201B310B80918F01CE
:101D80009091900197FF03C09195819591090597D6
:101D9000281739070CF079CF0E94680463E070E0DF
:101DA00080E090E00E949303B80182E00E949404D6
:101DB0006CCFEFE9F1E01382128288EE93E0A0E0AD
:101DC000B0E084839583A683B78383E191E0918318
:101DD000808385EC90E09587848784EC90E09787FA
:101DE000868780EC90E0918B808B81EC90E0938BE8
:101DF000828B82EC90E0958B848B86EC90E0978BC5
:101E0000868B118E128E138E148E0895EE0FFF1F87
:101E10000590F491E02D09945058BB27AA270E9401
:101E2000240F0C9497100E94891038F00E94901093
:101E300020F039F49F3F19F426F40C9486100EF428
:101E4000E095E7FB0C948010E92F0E94A81058F34E
:101E5000BA17620773078407950720F079F4A6F58F
:101E60000C94CA100EF4E0950B2EBA2FA02D0B0186
:101E7000B90190010C01CA01A0011124FF27591BCF
:101E800099F0593F50F4503E68F11A16F040A22FD5
:101E9000232F342F4427585FF3CF46953795279546
:101EA000A795F0405395C9F77EF41F16BA0B620B45
:101EB000730B840BBAF09150A1F0FF0FBB1F661F8C
:101EC000771F881FC2F70EC0BA0F621F731F841FCF
:101ED00048F4879577956795B795F7959E3F08F0F5
:101EE000B0CF9395880F08F09927EE0F97958795B7
:101EF00008950E945C1008F481E008950E94920FFA
:101F00000C9497100E94901058F00E94891040F095
:101F100029F45F3F29F00C94801051110C94CB10E0
:101F20000C9486100E94A81068F39923B1F35523EE
:101F300091F3951B550BBB27AA27621773078407DC
:101F400038F09F5F5F4F220F331F441FAA1FA9F372
:101F500035D00E2E3AF0E0E832D091505040E69560
:101F6000001CCAF72BD0FE2F29D0660F771F881FC1
:101F7000BB1F261737074807AB07B0E809F0BB0BB4
:101F8000802DBF01FF2793585F4F3AF09E3F5105C8
:101F900078F00C9480100C94CB105F3FE4F3983EE3
:101FA000D4F3869577956795B795F7959F5FC9F7B1
:101FB000880F911D9695879597F90895E1E0660F32
:101FC000771F881FBB1F621773078407BA0720F0AB
:101FD000621B730B840BBA0BEE1F88F7E095089514
:101FE0000E94B01088F09F5798F0B92F9927B751E9
:101FF000B0F0E1F0660F771F881F991F1AF0BA95AD
:10200000C9F714C0B13091F00E94CA10B1E0089530
:102010000C94CA10672F782F8827B85F39F0B93F22
:10202000CCF3869577956795B395D9F73EF490955F
:102030008095709561957F4F8F4F9F4F0895E894DD
:1020400009C097FB3EF490958095709561957F4F00
:102050008F4F9F4F9923A9F0F92F96E9BB279395AE
:10206000F695879577956795B795F111F8CFFAF4BE
:10207000BB0F11F460FF1BC06F5F7F4F8F4F9F4FEF
:1020800016C0882311F096E911C0772321F09EE84D
:10209000872F762F05C0662371F096E8862F70E0B3
:1020A00060E02AF09A95660F771F881FDAF7880F8D
:1020B0009695879597F90895990F0008550FAA0BE3
:1020C000E0E8FEEF16161706E807F907C0F012164B
:1020D0001306E407F50798F0621B730B840B950B4E
:1020E00039F40A2661F0232B242B252B21F40895A3
:1020F0000A2609F4A140A6958FEF811D811D089540
:1021000097F99F6780E870E060E008959FEF80ECAA
:10211000089500240A94161617061806090608954D
:1021200000240A9412161306140605060895092EB3
:102130000394000C11F4882352F0BB0F40F4BF2B22
:1021400011F460FF04C06F5F7F4F8F4F9F4F089562
:1021500057FD9058440F551F59F05F3F71F0479558
:10216000880F97FB991F61F09F3F79F0879508953D
:10217000121613061406551FF2CF4695F1DF08C05C
:10218000161617061806991FF1CF86957105610579
:1021900008940895E894BB2766277727CB0197F921
:1021A00008950E945C1008F48FEF089516F00C94C7
:1021B00093110C94861068940C9480100E94B010B7
:1021C000A8F39923C1F3AEF3DF93CF931F930F933B
:1021D000FF92C92FDD2788232AF02197660F771FEA
:1021E000881FDAF720E030E040E85FEB9FE38839B2
:1021F00020F0803E38F021968F770E940D0FEEEB95
:10220000F0E004C00E940D0FEBEEF0E00E94A1117F
:102210008B01BE01EC01FB2E6F5771097595771F7D
:10222000880B990B0E94211028E132E741E35FE31C
:102230000E943911AF2D9801AE01FF900F911F91AF
:10224000CF91DF910E94240F0C9497100E943911B6
:102250000C9497100E94891038F00E94901020F082
:10226000952311F00C9480100C94861011240C947A
:10227000CB100E94A81070F3959FC1F3950F50E00A
:10228000551F629FF001729FBB27F00DB11D639F28
:10229000AA27F00DB11DAA1F649F6627B00DA11DCE
:1022A000661F829F2227B00DA11D621F739FB00D74
:1022B000A11D621F839FA00D611D221F749F3327E4
:1022C000A00D611D231F849F600D211D822F762F7D
:1022D0006A2F11249F5750409AF0F1F088234AF05A
:1022E000EE0FFF1FBB1F661F771F881F91505040C6
:1022F000A9F79E3F510580F00C9480100C94CB10F0
:102300005F3FE4F3983ED4F3869577956795B7954C
:10231000F795E7959F5FC1F7FE2B880F911D969566
:10232000879597F908959F3F31F0915020F4879554
:1023300077956795B795880F911D9695879597F92D
:102340000895DF93CF931F930F93FF92EF92DF9245
:102350007B018C01689406C0DA2EEF010E943911CE
:10236000FE01E894A5912591359145915591A6F3EB
:10237000EF010E94240FFE019701A801DA9469F78A
:10238000DF90EF90FF900F911F91CF91DF91089513
:1023900081E090E0F8940C942812052E97FB1EF42F
:1023A00000940E94E41157FD07D00E94F71107FC2A
:1023B00003D04EF40C94E41150954095309521953E
:1023C0003F4F4F4F5F4F0895909580957095619561
:1023D0007F4F8F4F9F4F08950E941912A59F900D18
:1023E000B49F900DA49F800D911D11240895A1E22A
:1023F0001A2EAA1BBB1BFD010DC0AA1FBB1FEE1F7F
:10240000FF1FA217B307E407F50720F0A21BB30BC9
:10241000E40BF50B661F771F881F991F1A9469F745
:1024200060957095809590959B01AC01BD01CF01A1
:102430000895A29FB001B39FC001A39F700D811D9D
:102440001124911DB29F700D811D1124911D0895BD
:04245000F894FFCF2E
:102454000101010C00E8030000C04001000000007D
:1024640000000026025601A301810195016D0200BE
:00000001FF
